:020000040000FA
:02000000FC28DA
:08000800000000000000831657
:100010000130850011309F00FF23900083120330D0
:100020009F00851005110930900008006730B0006E
:100030005C30B1005130B2004830B3003430B4000D
:100040002E30B5002830B6002230B7001F30B8007F
:100050001030A7000030C100C400FF30C2000430DF
:10006000C3000800C00B32280800AF00C0000030F9
:10007000A800A900AB00AC00A400FF30A200270834
:10008000A00000088F008E009F149F1845281E08AE
:10009000A3000310A8070318A90A031024020318D9
:1000A00053282308A400230803102202031C5A2803
:1000B0002308A2002F08C00032209F149F185E283A
:1000C0001E08A3000310AB070318AC0A0310240298
:1000D00003186C282308A400230803102202031C21
:1000E00073282308A2002F08C00032209F149F18F5
:1000F00077281E08A3000314A802031CA9030314F5
:100100002402031885282308A400230803142202CC
:10011000031C8C282308A2002F08C00032209F1443
:100120009F1890281E08A3000314AB02031CAC0305
:100130000314240203189E282308A4002308031490
:100140002202031CA5282308A2002F08C0000230A9
:100150000314C0023220A00B4428A91FB628A90905
:10016000A80903100030A8070318A90AAC1FBF286C
:10017000AC09AB0903100030A8070318AC0A033020
:10018000A0000310A90CA80C0310AC0CAB0CA00B26
:10019000C128220803102402A5000310A50C28087A
:1001A00003102B02031CD8280310280C2B07DB2874
:1001B00003102B0C280703102502031CE128003034
:1001C000E2280130AE000800380835202E08031957
:1001D000EF28C30BEF2805151030C300C4004408F6
:1001E000031DC40BF4280511080085140A303220C1
:1001F00085100A303220F528072016204108031DFB
:1002000064294208C500E420330835202E08031D68
:100210000C29C50B0329FE28350835202E08031D9F
:100220001429C50B0329FE284208C500E420300824
:1002300035202E08031D1F29C50B1629FE28350859
:1002400035202E08031D2729C50B1629FE28420834
:10025000C500E420360835202E08031D3229C50BC1
:100260002929FE28310835202E08031D3A29C50BFF
:100270002929FE284208C500E420330835202E082D
:10028000031D4529C50B3C29FE28350835202E08BD
:10029000031D4D29C50B3C29FE284208C500E4205A
:1002A000360835202E08031D5829C50B4F29FE2876
:1002B000300835202E08031D6029C50B4F29FE2864
:1002C0000130C1008514FE284208C500E42033082F
:1002D00035202E08031D6F29C50B6629FE28350819
:1002E00035202E08031D7729C50B6629FE284208F4
:1002F000C500E420320835202E08031D8229C50BD5
:100300007929FE28350835202E08031D8A29C50BBA
:100310007929FE284208C500E420310835202E083E
:10032000031D9529C50B8C29FE28340835202E087D
:10033000031D9D29C50B8C29FE284208C500E42019
:10034000320835202E08031DA829C50B9F29FE2839
:10035000340835202E08031DB029C50B9F29FE281F
:100360004208C500E420300835202E08031DBB29B3
:10037000C50BB229FE28340835202E08031DC329D9
:0E038000C50BB229FE280030C1008510FE28F2
:00000001FF
